:1000000033C04FC04EC04DC04CC04CC04AC049C0A8
:1000100048C047C046C045C044C043C042C0010AB2
:100020002A4B7A85FF0102030507EEF3F400010273
:1000300003050700070503020100020407EEF3F4BD
:10004000F000020407000704020001020306EEF3B9
:10005000F4F000010203060006030201000203059A
:1000600007000704EE00070011241FBECFE5D1E012
:10007000DEBFCDBF20E0A0E6B0E001C01D92A137F9
:10008000B207E1F7E2E7F0E01282108688E58187A7
:10009000E0E6F0E08DEF87838EEF8583712CA1D0B1
:1000A0003CC1AECF189525B7277E25BF29B7226062
:1000B00029BF21E022BF019728F020E18895215037
:1000C000E9F7F9CF089588EE93E0EDCF369A3699A7
:1000D000FECF85B1089580917100EEE7F0E0808356
:1000E000818382830895CF93C72D81E0870D8F731D
:1000F000782E662D90E003D16FEF8C2F90E0CF919A
:10010000FEC0FF920F931F93CF93DF93F82E03E768
:1001100010E0CEE7D0E0F11005C0CE01E8D0F80144
:10012000808304C0F8016081CE01E9D021970F5F80
:100130001F4FC537D10579F7DF91CF911F910F91EF
:10014000FF900895D0DF81E0DCCFEF92FF920F9314
:100150001F93CF93C82F8B018EE1E82E80E0F82EFD
:10016000CC2361F0F701849189BDC8019CDF19BCE3
:10017000C80199DFC80197DFC150F2CFCF911F911D
:100180000F91FF90EF900895CF93DF93D82F64E104
:1001900070E08AE0DADF84EF91E085DF8D2F64E69E
:1001A0009AD0CAE06C2F97D0892F68EC70E0CDDF31
:1001B0008ADF8D2F6C2F8FD0D92F8DD0892F68ECAF
:1001C00070E0C3DF80DF68EC70E08D2FBEDF7BDF87
:1001D00064E170E08AE0B9DF84EF91E0DF91CF91D4
:1001E00062CF10927100712C872D90E080D0682E24
:1001F0008F3F31F08FEF68120AC0612CA3DF09C076
:10020000872D91E0970D792E803470F3F3CF80E045
:1002100078DF80917A008F5F90E045E250E088239C
:1002200099F09A012F5F3F4FF9013197E491A92F7F
:10023000B0E0A859BF4FEC93EE2319F0922F941B16
:10024000F1CF8150A901EBCF90937C0090937D007A
:10025000862D853FE0F42091800030917F002313AC
:100260002DC030917E00231329C02F3F71F533DF5D
:1002700080917E008F5F80937E0080917F008F5FF2
:1002800080937F00809180008F5F809380008FE358
:1002900084BB81E087BB9AEF98BB83BF81E88ABDAE
:1002A00085B7806285BF789481EA87B986EC86B984
:1002B0008CE291E0F8DE0ADF67DFFACF0CDF809195
:1002C00074008111E4CF612CE2CF8F5F682E891713
:1002D00078F2612CCDCF991B79E004C0991F961755
:1002E00008F0961B881F7A95C9F780950895E199C3
:1002F000FECF1FBA8EBBE09A99278DB30895262FA3
:10030000E199FECF1CBA1FBA8EBB2DBB0FB6F89475
:0E031000E29AE19A0FBE01960895F894FFCF8D
